:1000000098C00000BEC00000BCC00000BAC0000024
:10001000B8C00000B6C00000B4C000000C94AB1023
:10002000B0C00000AEC00000ACC00000AAC000001C
:10003000A8C00000A6C00000A4C00000A2C000002C
:100040000C9441139EC000000C948C110C94C611AA
:1000500098C0000096C0000094C0000092C000004C
:1000600090C000008EC000000000000000000000F2
:100070000000000000000000000000000000000080
:100080000000000000000000000000000000000070
:100090000000000000000000000000000000000060
:1000A0000000000000000000000000000000000050
:1000B0000000000000000000000000000000000040
:1000C0000000000000000000000000000000000030
:1000D0000000000000000007000201000003040609
:1000E0000000000000000000010204081020408011
:1000F0000102040810200102040810200404040472
:1001000004040404020202020202030303030303C1
:100110000000000023002600290000000000250048
:1001200028002B0000000000240027002A00E51012
:10013000801211241FBECFEFD8E0DEBFCDBF11E08B
:10014000A0E0B1E0ECEFFDE202C005900D92A03915
:10015000B107D9F727E0A0E9B1E001C01D92A733AC
:10016000B207E1F711E0C2E3D1E004C02297FE013B
:100170000E94F816CE32D107C9F70E941C0E0C94CB
:1001800050143ECF4F925F926F927F928F929F92C8
:10019000AF92BF92CF92DF92EF92FF920F931F9395
:1001A000CF93DF93EC01C42E8AA1841304C08BA1EA
:1001B000681709F479C0CAA26BA31C2D6C1508F44A
:1001C000162FFE0180E090E021E01C1102C0208388
:1001D00001C010820196319680329105B1F711234A
:1001E00009F462C081E088836C2D70E080E090E0CB
:1001F0000E9454154B015C01612F70E080E090E09B
:100200000E9454159B01AC01C501B4010E94BB14AE
:10021000962E872E782E692EA12CB12C00E010E0AE
:10022000D12CE12CF12C5524539430C06A2D7B2D18
:10023000802F912F0E942315462E7727882777FD40
:100240008095982F0E9456159B01AC016A2D7B2D3D
:10025000802F912F0E94521420E030E040E05FE3B5
:100260000E94061687FF4394FE01E40DF11D5082A3
:10027000B401C301272F382D492F562D6A2D7B2D10
:10028000802F912F0E9453145B018C01C701B6018E
:100290000E9456159B01AC016A2D7B2D802F912F5A
:1002A0000E94B71487FDC2CFDF91CF911F910F91AC
:1002B000FF90EF90DF90CF90BF90AF909F908F9086
:1002C0007F906F905F904F900895FC0121A1E20F05
:1002D000F11D80810895FC0141A1242F30E082A10D
:1002E00090E00197281739071CF44F5F41A3089548
:1002F00011A20895FC0171836083EE5DFC4F1082B2
:100300000895CF92DF92EF92FF920F931F93CF93B6
:10031000FC01EE5DFC4F50815F3908F042C0752F43
:100320007E5FC72F19C0FD013197EE0FFF1FEE0F43
:10033000FF1FE80FF91FC280D380E480F580AA0F69
:10034000BB1FAA0FBB1FA80FB91F1296CD92DD923B
:10035000ED92FC921597C150AC2FB0E0109719F7B1
:100360000AC0E80FF91FDF01AF57BD4FAC91EE5740
:10037000FD4FA0837150E72FF0E0309791F7FC011B
:100380000283138324833583EE57FD4F20E1629F60
:10039000B0011124642B6083FC01EE5DFC4F5F5FB4
:1003A0005083CF911F910F91FF90EF90DF90CF90EE
:1003B00008950F931F93FC01EE5DFC4FA08166230F
:1003C00001F1B0E018C0FB013196EE0FFF1FEE0FF8
:1003D000FF1FE80FF91F0281138124813581FB0182
:1003E000EE0FFF1FEE0FFF1FE80FF91F02831383AD
:1003F000248335834F5F642F70E0A617B7071CF77F
:1004000020C0AE5F50E018C0FB013197EE0FFF1F18
:10041000EE0FFF1FE80FF91F028113812481358140
:10042000FB01EE0FFF1FEE0FFF1FE80FF91F028306
:10043000138324833583A1506A2F70E04617570732
:100440001CF31F910F910895FC01EE5DFC4F662394
:10045000A1F0608170E00BC0280F391FF901ED5742
:10046000FD4F5081F901EE57FD4F50834F5F242F10
:1004700030E06217730784F7089560816E5F50E083
:100480000BC0280F391FF901EF57FD4F7081F9019B
:10049000EE57FD4F70836150262F30E0421753070F
:1004A00084F308959F92AF92BF92CF92DF92EF9222
:1004B000FF920F931F93CF93DF93EC016A017B01AF
:1004C00088819981892B09F448C0FE01ED5DFC4FBC
:1004D0004083518362837383FE01EE5DFC4F808114
:1004E000811135C03AC0E92DF0E0DE0184E0989E2C
:1004F000A00DB11D112412960D911D912D913C91CD
:100500001597C016D106E206F306F8F0EC0FFD1FB2
:10051000EE57FD4F9081892F82958F70692F617002
:1005200091FD626092FD646093FD6860E881F981ED
:100530000995492D61E0CE013CDF492D61E0CE01F6
:1005400083DFF501808181508083939402C0912CD8
:100550005F01F5018081981630F2DF91CF911F91F4
:100560000F91FF90EF90DF90CF90BF90AF909F9052
:100570000895CF92DF92EF92FF920F931F93CF9344
:10058000DF939091BE01911130C090E2899F80016C
:100590001124C5E0D1E080E1C82E81E0D82E780199
:1005A000ECE0EE0EF11CFE0131974081B80183E8CA
:1005B00096E00E94EE10B8016F5F7F4F488183E89C
:1005C00096E00E94EE10F60141916F01B70183E8B9
:1005D00096E00E94EE100E5F1F4F2296FFEFEF1A7B
:1005E000FF0A81E0C131D807F1F6DF91CF911F9169
:1005F0000F91FF90EF90DF90CF900895AF92BF9250
:10060000CF92DF92EF92FF920F931F93CF93DF93DE
:100610001F92CDB7DEB7482F80E2489F800111249A
:1006200095E0A92E91E0B92E7801ECE0EE0EF11CD8
:1006300020E1C22E21E0D22EB80183E896E0498362
:100640000E94EC10F50131978083B8016F5F7F4FF6
:1006500083E896E00E94EC10F5018083B70183E8FF
:1006600096E00E94EC10F60181936F010E5F1F4F20
:10067000F2E0AF0EB11C8FEFE81AF80A4981E1E110
:10068000AE16E1E0BE06C1F667EE73E083E896E0E1
:100690000F90DF91CF911F910F91FF90EF90DF901E
:1006A000CF90BF90AF900C94EE10EF92FF920F930B
:1006B0001F93CF93DF93E12CFF24F3948E2D9EDFC5
:1006C00048E551E0C4E0D1E0A5E0B1E028E630E043
:1006D00060E171E04F5F5F4FF9010591149108836C
:1006E000F9013196059114910C93FB01F192BF0130
:1006F000229612962E5F3F4FF1E04E355F0751F77D
:100700008E2D37DFE39486E0E812D8CFDF91CF91CA
:100710001F910F91FF90EF90089568EE73E083E8CA
:1007200096E00E94EC10853081F469EE73E083E876
:1007300096E00E94EC10863041F46AEE73E083E8A4
:1007400096E00E94EC108730E9F0AFDF40E067EE02
:1007500073E083E896E00E94EE1045E068EE73E0F7
:1007600083E896E00E94EE1046E069EE73E083E8CD
:1007700096E00E94EE1047E06AEE73E083E896E0B0
:100780000C94EE1008959A01AB01682F8FE396E068
:100790000C94EA0E4F925F926F927F928F929F928B
:1007A000AF92BF92CF92DF92EF92FF920F931F937F
:1007B000CF93DF93C82FD62F042F8FE396E00E94AC
:1007C000A510C090B501D090B601E090B701F090AF
:1007D000B8016C197D098E099F09693E7340810536
:1007E000910508F44CC18FE396E00E94A510C090DB
:1007F000BA01D090BB01E090BC01F090BD016C1932
:100800007D098E099F09653671058105910508F4FA
:1008100036C11092B901EC2FF0E0DF01A05FBE4FAE
:100820008C91D1116CC010E0833019F4EE0FFF1FD2
:1008300072C030E1832E31E0932E800E911EF401C0
:100840008081853009F01BC1000F111F0C5F1E4F06
:10085000D8011196AC90B12C00901C0102C0B59447
:10086000A7940A94E2F7BFEFAB1ABB0AF801F08035
:100870006C2F8FE396E00E942B0ED82F2F2D30E0A7
:10088000D5010E94E016C12CD12C7601CA94A70193
:1008900096010E94B91629013A012D2F30E0D501A9
:1008A0000E94E016A70196010E94B916421653064F
:1008B0006406750611F1D80111960C9110E0D4016F
:1008C000EC91F0E0E95EFE4F008002C015950795BF
:1008D0000A94E2F76C2F8FE396E00E942B0E282FEC
:1008E00030E0D8010E94E016A70196010E94B916D7
:1008F0002F5F3F4F4F4F5F4F8BC0F401ABC0813034
:1009000029F0853019F0843009F044C010E0EE0F72
:10091000FF1FED0FF11DEC5FFE4FE080F12C005F3B
:100920001E4FD801EC91F0E0E95EFE4F008002C05E
:10093000F594E7940A94E2F76C2F8FE396E00E9417
:100940002B0EF801608190E0E62FF0E0E95EFE4FAB
:10095000008002C0959587950A94E2F7E816F9069B
:1009600009F479C06C2F8FE396E00E942B0E90E083
:10097000D801EC91F0E0E95EFE4F008002C0959551
:1009800087950A94E2F7019683709927892B09F0DD
:1009900049C046C0823009F072C010E0F801EE0F85
:1009A000FF1FEC5FFE4FF1806C2F8FE396E00E94FB
:1009B0002B0ED82F2F2D30E0A9E0B0E00E94D416E6
:1009C000C12CD12C7601CA94A70196010E94B916B8
:1009D00049015A012D2F30E0A9E0B0E00E94D41661
:1009E000A70196010E94B91682169306A406B506C1
:1009F00071F16C2F8FE396E00E942B0E282F30E0D0
:100A0000A9E0B0E00E94D416A70196010E94B91691
:100A10002370332744275527232B242B252B11F410
:100A200067E001C060E08FE396E00E94A10E8FE3D3
:100A300096E00E94A5106093BA017093BB01809369
:100A4000BC019093BD0181E08093B90118C0F80109
:100A5000E05FFE4F60818FE396E0DF91CF911F91C1
:100A60000F91FF90EF90DF90CF90BF90AF909F904D
:100A70008F907F906F905F904F900C94A10EDF91BC
:100A8000CF911F910F91FF90EF90DF90CF90BF908B
:100A9000AF909F908F907F906F905F904F90089550
:100AA000E0911601F0E0DF01A05FBE4F8C9190E075
:100AB000EE0FFF1FEC5FFE4FDC01A85ABE4F2C91DA
:100AC0002083DC01A05ABE4F8C91818308951F932F
:100AD000CF93DF93C82F811150C060E08FE396E081
:100AE0000E94E50E882369F181E080933E02C5E013
:100AF000D1E010E04881612F8FE396E00E94430F20
:100B000022961F5F1630B1F78091AF018823C9F09C
:100B10008091BF012EDD1092AF018FE396E00E941D
:100B2000A5106093B0017093B1018093B2019093CE
:100B3000B3018FEF8093160160E08FE396E00E948F
:100B4000A10E60E08FE396E00E94E50E81116AC07D
:100B500010923E02C4E0D1E010E04881612F8FE3A3
:100B600096E00E94430F22961F5F1630B1F78091E6
:100B7000AF01882309F456C00EC0813009F052C07D
:100B800061E08FE396E00E94E50E81114BC08091F9
:100B9000AF018823B1F08091BF01EBDC1092AF016F
:100BA0008FE396E00E94A5106093B0017093B101AD
:100BB0008093B2019093B3018FEF8093160160E0B0
:100BC0002AC080913E0281112DC0E0911601EF3FB5
:100BD00049F18091BE01811118C0F0E0E05FFE4F45
:100BE0008081873018F48F5F808301C0C08358DF15
:100BF00060911601E62FF0E0EE0FFF1FEC5FFE4F55
:100C000040818FE396E00E94430FE0911601F0E0EF
:100C1000E05FFE4F60818FE396E0DF91CF911F91FF
:100C20000C94A10EDF91CF911F9108952F923F92C6
:100C30004F925F926F927F928F929F92AF92BF92EC
:100C4000CF92DF92EF92FF920F931F93CF93DF9398
:100C500000D000D000D0CDB7DEB7282E90E09E8324
:100C60008D83880F991F9A838983FC01EC5FFE4F67
:100C7000808190E0ED81FE81E05FFE4FE081F0E059
:100C8000E95EFE4F008002C0959587950A94E2F7D1
:100C9000382E3394A981BA81AA53BE4FBC83AB834B
:100CA0008D919C91892B09F46FC08FE396E00E948F
:100CB000A5106B017C010D811E81000F111F000F1B
:100CC000111FF801EA5DFD4F408051806280738002
:100CD000832C912CA12CB12CF801E252FE4F808183
:100CE0009181A281B381C81AD90AEA0AFB0AC30119
:100CF000B201A50194010E9497162C153D054E05E1
:100D00005F0508F041C0E981FA81EE52FE4F808113
:100D10009181019691838083EB81FC81E080F18059
:100D2000832D90E08E159F0519F0A32DAE1901C0FB
:100D3000A0E02EEDC22E21E0D22EC00ED11EB0E0DA
:100D4000A30192010E94E616A50194010E94971644
:100D5000F801EA50FE4F80819181A281B381280F72
:100D6000391F4A1F5B1FD6012D933D934D935C9312
:100D70001397ED81FE81EE0FFF1FEA53FE4FB1E0A6
:100D8000EB1AF108F182E0820D811E8100541E4FA2
:100D9000F80180818823A9F18FE396E00E94A510D5
:100DA0006B017C012D813E81220F331F220F331FE7
:100DB000F901E25FFD4F80819181A281B381C81A60
:100DC000D90AEA0AFB0AF901EA5DFD4F232D30E05A
:100DD00040E050E060817181828193810E9497168A
:100DE00056954795379527952C153D054E055F057A
:100DF00040F440E050E061E070E0822DC4DCD801B6
:100E00001C920D811E81000F111F0E521E4FF80102
:100E100080819181892B19F1ED81FE81E054FE4F93
:100E200081E0808340E050E060E070E0822DABDC48
:100E30008FE396E00E94A510ED81FE81EE0FFF1F6B
:100E4000EE0FFF1FE25FFD4F608371838283938308
:100E5000D8018D919C91119701978D939C93269623
:100E60000FB6F894DEBF0FBECDBFDF91CF911F91BB
:100E70000F91FF90EF90DF90CF90BF90AF909F9039
:100E80008F907F906F905F904F903F902F9008953C
:100E90000F931F9380911F0190912001A091210138
:100EA000B0912201BC0155274427482759276A27BA
:100EB0007B27DB01CA01E5E0B695A7959795879555
:100EC000EA95D1F784279527A627B72740912301D4
:100ED00050912401609125017091260140931F01DA
:100EE000509320016093210170932201009127010A
:100EF000109128012091290130912A0100932301AA
:100F000010932401209325013093260104271527EF
:100F100026273727082719272A273B27880F991FB5
:100F2000AA1FBB1F082719272A273B270093270141
:100F3000109328012093290130932A01B801C90197
:100F40001F910F910895CF93DF93EC01A1DF9B01D7
:100F5000AC0144275527DE010E94F016AC0166273C
:100F60007727CA01DF91CF9108952F923F924F9238
:100F70005F927F928F929F92AF92BF92CF92DF92B9
:100F8000EF92FF920F931F93CF93DF9300D0CDB7D3
:100F9000DEB7782E282E312CF101E05FFE4F8081E4
:100FA000833009F478C148F49101220F331F813056
:100FB00009F449C008F0C7C00CC0853009F4BCC2B0
:100FC00008F47CC2863009F4D1C1873009F0DDC253
:100FD000F5C1672D8FE396E029833A834AD72981AB
:100FE0003A81F901EC5FFE4F882379F0818190E02E
:100FF000880F892F881F990B892B09F0C6C2408161
:1010000020E1429FA001112405C0408180E1489F5A
:10101000A00111244F5F5F4F60E070E0872D0F90BB
:101020000F90DF91CF911F910F91FF90EF90DF9084
:10103000CF90BF90AF909F908F907F905F904F9098
:101040003F902F90A0CBF901EE52FE4F808191810D
:10105000019691838083B4E0CB2EB1E0DB2EC20EEB
:10106000D31ED60111966C9170E00090180102C059
:10107000759567950A94E2F76F5F6093AE0170E033
:101080000E948316892B09F080C211821082220CE3
:10109000331C220C331CAEE0EA2EA2E0FA2EE20C46
:1010A000F31C81010A5D1D4FF80180819181A281AD
:1010B000B381F70180839183A283B3838FE396E0AA
:1010C0000E94A510D8016D937D938D939C931397E7
:1010D0004091AE0181010A561E4FF601A0814130B8
:1010E00071F4F4E0AF9FC0011124AA2797FDA095E9
:1010F000BA2FF80180839183A283B3831AC0F701CA
:10110000C080D180E280F3809B01AC012C193D09A5
:101110004E095F09B0E00E94E6162FEF30E040E094
:1011200050E00E94B916D8012D933D934D935C93E6
:1011300013978FE396E00E94A5108B019C01F101AB
:10114000EA56FE4F9EC142EDC42E41E0D42EC20E9F
:10115000D31EF601008111810F5F1F4F11830083A1
:1011600054E0E52E51E0F52EE20EF31ED701119664
:101170002C9130E0A9E0B0E00E94D416812C912C93
:1011800054018A94A50194010E94B916622F2093FC
:10119000AE01211107C0F7014081F0E14F9FA0018E
:1011A000112438CFC80170E00E948316892B09F002
:1011B000ECC1D6011D921C928101000F111F000F7E
:1011C000111F8EE0C82E82E0D82EC00ED11E96E2EE
:1011D000492E92E0592E400E511EF20180819181DC
:1011E000A281B381F60180839183A283B3838FE3CD
:1011F00096E0ABD7D2016D937D938D939C9313971B
:10120000F101E054FE4F208131E02327208336E9AD
:10121000232E31E0332E200E311E222361F1F701FF
:10122000A081F60100811181228133816B017C0153
:10123000C01AD10AE20AF30AA7019601B0E00E949F
:10124000E616A50194010E94B916D1012D933D9394
:101250004D935C9313978FE396E077D78B019C01B6
:10126000F10180819181A281B381080F191F2A1F8A
:101270003B1F41E00FC18FE396E067D78B019C01D4
:10128000F10180819181A281B381080F191F2A1F6A
:101290003B1F40E0FFC08101000F111FF801EC5F10
:1012A000FE4F808190E000901A0102C095958795CD
:1012B0000A94E2F7D82ED3948FE396E046D7220C17
:1012C000331C220C331CF101EA5DFD4FA6EFEA2E20
:1012D000A1E0FA2EE20CF31CD7018D909D90AD9009
:1012E000BC90681979098A099B096083718382839C
:1012F00093838FE396E029D7F7016083718382831C
:1013000093838FE396E021D7F101E252FE4F608391
:10131000718382839383F801EE52FE4FD801AA5362
:10132000BE4F808191812D913C911197820F931F27
:101330002D2D30E0215031092D933C93019691835E
:101340008083872D0F900F90DF91CF911F910F9188
:10135000FF90EF90DF90CF90BF90AF909F908F90D5
:101360007F905F904F903F902F9060CCF101EE0FF7
:10137000FF1FEC5FFE4F81818F3F09F006C1C10165
:10138000880F991F880F991F9C01225F3D4F8C0188
:101390000A5D1D4FF80180819181A281B381F9011D
:1013A00080839183A283B3838FE396E0CED6D80166
:1013B0006D937D938D939C931397E7C07101EE0C11
:1013C000FF1C87010C5F1E4FF80181818F3F09F0E0
:1013D0006AC05101AA0CBB1CAA0CBB1C9EE0C92E02
:1013E00092E0D92ECA0CDB1C26E2822E22E0922E3D
:1013F0008A0C9B1CF40180819181A281B381F6014A
:1014000080839183A283B3838FE396E09ED6D40139
:101410006D937D938D939C93139736E9832E31E0E2
:10142000932E8A0C9B1CF801A081F601008111818A
:10143000228133815B016C01A01AB10AC20AD30A6E
:10144000A6019501B0E00E94E6162FEF30E040E0E3
:1014500050E00E94B916D4012D933D934D935C93B7
:101460001397F701EE52FE4F80819181019691838F
:10147000808380FF15C08FE396E067D68B019C01C7
:10148000F40180819181A281B381080F191F2A1F65
:101490003B1F42E0672D87E193E00E94810175C008
:1014A0004AE050E0B9CD8FEF90E04DDDD8012C91AE
:1014B00030E0281739070CF468C0F2CFF101EE0FC5
:1014C000FF1FEC5FFE4FC180D12C00901B0102C0BA
:1014D000D594C7940A94E2F7C394E12CF12CD12C53
:1014E0004F0113E1A12EBB24B39422C08FE396E0F9
:1014F0002CD68B019C01F4018081A501481B510968
:10150000E49EC001E59E900DF49E900D1124AA2743
:1015100097FDA095BA2F080F191F2A1F3B1F42E005
:10152000672D87E193E00E948101FFEFEF1AFF0A28
:10153000EC14FD04DCF229C084E2829D8001839DCD
:10154000100D1124015C1D4FC8010E946501882304
:1015500031F04AE050E060E070E0872D14D9C80116
:101560000F900F90DF91CF911F910F91FF90EF900F
:10157000DF90CF90BF90AF909F908F907F905F90C3
:101580004F903F902F900C946B010F900F90DF9134
:10159000CF911F910F91FF90EF90DF90CF90BF9070
:1015A000AF909F908F907F905F904F903F902F9043
:1015B00008954F925F926F927F92BF92CF92DF9287
:1015C000EF92FF920F931F93CF93DF93B82E082FC4
:1015D00010E0F801EE0FFF1FEC5FFE4F7180000F6F
:1015E000111F000F111F80819FEF791212C0F801A7
:1015F000EA5DFD4FC081D181C80FD11DF801E25FC6
:10160000FD4F80819181C81BD90B7E01F694E79430
:1016100036C0C1E0D1E0C81BD10993E0CC0FDD1F7B
:101620009A95E1F7BE0180E090E00E94541520E019
:1016300030E040E05AE30E940A166B017C01E8E0CA
:101640007E9EB0011124882777FD8095982F0E94F7
:1016500056159B01AC01C701B6010E940A160E94F3
:1016600023157B016C177D0720F07E01F1E0EF1A56
:10167000F108E114F10419F4EE24E394F12C8FE362
:1016800096E063D50A501E4FF80140805180628079
:10169000738064197509860997092E01612C712CD4
:1016A0006415750586059705D0F08FE396E04DD556
:1016B000F8016083718382839383A70160E070E007
:1016C0008B2DDF91CF911F910F91FF90EF90DF90C5
:1016D000CF90BF907F906F905F904F9054C8DF91F4
:1016E000CF911F910F91FF90EF90DF90CF90BF901F
:1016F0007F906F905F904F900895E82FF0E0E05F4B
:10170000FE4F9081933019F0963019F401C08ECAC3
:1017100050CF0895811105C028DC81E026DC82E0ED
:1017200005C0813021F484E020DC85E01ECC0895E2
:10173000CF93C82F811102C080E0ECDF80913E067C
:101740008C1304C084E011DC85E00FDC8EEF90E0A8
:10175000FADB2091950130E08217930724F081E0B5
:1017600080933E0602C010923E06CF9108956130EC
:1017700071F040F0623019F06330A1F40BC04AE020
:1017800050E00CC040E050E061E070E009C040E093
:1017900050E004C090E4499FA001112460E070E093
:1017A0000C94C303089540E0E2CF40E056E960E0C6
:1017B00070E084E896E025D662E571E084E896E082
:1017C0004ED762E086E00E94F01386E00E94281463
:1017D000892B19F481E08093BE0148E95BE067E65C
:1017E00075E08FE396E07AD263ED7BE087E193E0EA
:1017F0000E947A010E948D0367EE73E083E896E011
:10180000EBD48093BF010C94FE022F923F924F9233
:101810005F926F927F928F929F92AF92BF92CF9280
:10182000DF92EF92FF920F931F93CF93DF9300D03D
:1018300000D000D0CDB7DEB78FE396E086D46B0141
:101840007C0160E08FE396E0C0D2882309F4BBC13D
:1018500061E08FE396E0B9D28111BEC1B4C181E0ED
:101860008093AF018091AF01811110C0B701A60133
:1018700087E193E00E945202809116018093B401A7
:1018800005E011E07801A12CB12C51C080919101AB
:1018900090919201A0919301B0919401A7019601BA
:1018A000281B390B4A0B5B0BDA01C9018D329140C1
:1018B000A105B105B8F0C0929101D0929201E092D9
:1018C0009301F092940180919001873020F48F5F12
:1018D0008093900102C010929001609190018FE37B
:1018E00096E02FD210E00FEF612F8FE396E0FCD24D
:1018F0008823C9F08091BF010E94B9021093BF01F3
:10190000812F0E94FE021092AF01C092B001D092CE
:10191000B101E092B201F092B3010093160160E0D0
:101920008FE396E00ED21F5F1630F1F69FCF43E0B3
:10193000A416B10409F46EC0DA2C8A2DDEDE809183
:101940003E026A2D8823F9F08FE396E0C3D281111D
:1019500039C040911601842F90E0A816B90641F4D1
:101960008091AF01811104C061E08A2D0E94CA03F9
:101970008091BE01811126C06D2D8FE396E06BD161
:10198000D7018C931FC08FE396E0A4D281111AC0B7
:1019900040911601842F90E08A159B0541F48091B7
:1019A000AF01811104C060E08A2D0E94CA038091BA
:1019B000BE01811107C06D2D8FE396E04CD1F70178
:1019C000319780836D2D8FE396E08ED2882311F1BD
:1019D000D09216018091B4018D1559F08FE396E0F5
:1019E000B4D36093B5017093B6018093B70190931F
:1019F000B8018091B90181110DC08091AF018111B1
:101A000009C0E0911601F0E0E05FFE4F60818FE3D6
:101A100096E097D1BFEFAB1ABB0AE2E0EE0EF11CE5
:101A2000F6E0AF16B10409F082CF63E08FE396E0F1
:101A300012D18093950150E1E52E51E0F52E64E03E
:101A4000A62E61E0B62E1E821D82412C512C320141
:101A50004A94E4E23E2E8D80D7018C91853009F0C6
:101A60009FC0F801C080D12C00901C0102C0D59409
:101A7000C7940A94E2F7FFEFCF1ADF0AD5012C9042
:101A8000682D8FE396E0E7D0982E222D30E0D60126
:101A90000E94E016A30192010E94B91629833A839D
:101AA0004B835C83292D30E0D6010E94E016A30110
:101AB00092010E94B91689819A81AB81BC818217FB
:101AC0009307A407B50741F1D8018C9190E0D701A5
:101AD000EC91F0E0E95EFE4F008002C0959587959D
:101AE0000A94E2F7DC011296F5012081D82ED394F6
:101AF00030E00E94E016A30192010E94B9164D81C8
:101B00005E81349EC001359E900D11244D2D622FB3
:101B1000815C9D4F0E94C200D801CC90D12CD7018E
:101B2000EC91F0E0E95EFE4F008002C0D594C794CE
:101B30000A94E2F7682D8FE396E08DD0D701EC91FF
:101B4000F0E0E95EFE4F208190E0022E02C0959504
:101B500087950A94E2F7C816D90611F1F801808139
:101B600090E002C0959587952A95E2F7DC011296E0
:101B7000F5012081D82ED39430E00E94E016A30115
:101B800092010E94B9164D815E81349EC001359E3E
:101B9000900D11244D2D622F815C9D4F0E94C2003B
:101BA0008D819E8101969E838D839FEFE91AF90AAC
:101BB0000E5F1F4FA2E0AA0EB11CED81FE81369789
:101BC00009F049CF20C0C092B001D092B101E0929B
:101BD000B201F092B30146CE8091B0019091B10173
:101BE000A091B201B091B301A7019601281B390B56
:101BF0004A0B5B0BDA01C90189389341A105B10594
:101C000008F02DCE2FCE26960FB6F894DEBF0FBE6D
:101C1000CDBFDF91CF911F910F91FF90EF90DF909B
:101C2000CF90BF90AF909F908F907F906F905F907C
:101C30004F903F902F9008956ED5B7DDE6DDFECF33
:101C400008950895089580E00895089508950895E9
:101C500081E008950895860F911D860F911DFC0166
:101C6000858508955D9A5D980895882311F05B9AA3
:101C700008955B98089580E480937C00EAE7F0E0A3
:101C800080E880838081876080830895ECE7F0E0BE
:101C90009081907790839081982B908321E030E021
:101CA000082E01C0220F0A94EAF720937E000895BF
:101CB000EAE7F0E0808180648083089580917A0073
:101CC0008295817008952091780030917900932F4A
:101CD00080E0AC01422B9A01C9010895CF93DF93B4
:101CE000EC01F894539A559A549A5D985C985298DE
:101CF000579822982198209A259A5A9A5F9A2A9A58
:101D0000299A289A7DA76CA75FA74EA782E08093A7
:101D1000B000E0E7F0E080818260808387E080931C
:101D2000B1008093B3001092B200A5DF1BA680E043
:101D3000ADDFBEDF8FEF8E831F827894DF91CF916E
:101D40000895FC01A62FB0E0AF5CBE4F8C9180FDE2
:101D500002C0289A01C0289890A981FD02C0906411
:101D600001C09F7B90AB90A982FD02C0906801C02A
:101D70009F7790AB0895CF93DF93EC01ECA5FDA581
:101D8000309791F089859B85981719F08B8780E0B3
:101D900009958A859C85981739F08C87ECA5FDA557
:101DA00081E0DF91CF910994DF91CF91089523B124
:101DB00031E022FB222720F92327FC01218723B1D0
:101DC0002695217023272287D6CF860F911DFC01EF
:101DD00083850895CF93DF93FC01C62F673008F009
:101DE00045C0DC01A60FB11DA60FB11DD3963C93D3
:101DF0002E93D2974115510539F5D0A9232B91F493
:101E000081E090E0A0E0B0E0062E04C0880F991FAA
:101E1000AA1FBB1F0A94D2F7D82BD0AB91A9982B3D
:101E200091AB24C041E050E060E070E004C0440F9A
:101E3000551F661F771FCA95D2F7D42BD0AB40959C
:101E400081A9842381AB12C04130510579F441E06E
:101E500050E060E070E004C0440F551F661F771F1C
:101E6000CA95D2F7409580A9842380ABDF91CF91AA
:101E70000895FC0180A990E002C0959587956A9528
:101E8000E2F781700895262FFC01E60FF11D45A3AE
:101E900041E050E060E070E004C0440F551F661F51
:101EA000771F2A95D2F7FC012681242B26830895DB
:101EB000262F41E050E060E070E004C0440F551F61
:101EC000661F771F2A95D2F74095FC0126812423AF
:101ED00026830895FC01868190E002C09595879540
:101EE0006A95E2F781700895FC01878190E002C055
:101EF000959587956A95E2F781700895461718F0D1
:101F0000621738F004C0261710F480E0089581E0CD
:101F100008956417D0F3FBCF0F931F93CF93DF93F4
:101F2000EC01CCDE882309F464C08BA58E01080F78
:101F3000111D080F111DF80185859685928F818FDF
:101F4000C2DE9695879596958795F8019687858741
:101F5000ABA5FE01EA0FF11DEA0FF11D818D928DF7
:101F600025853685821B930B97FF03C0919581953C
:101F700091092F8141E050E060E070E00A2E04C03A
:101F8000440F551F661F771F0A94D2F7029734F04B
:101F9000422B4F836A2FCE018BDF03C04095422333
:101FA0004F831BA5812F90E0FC01EE0FFF1FEC0F6C
:101FB000FD1FDE01A80FB91F2585418D95966C91F7
:101FC000CE019CDF882319F0612FCE0171DF8BA534
:101FD0008F5F863010F48BA701C01BA6EBA5F0E045
:101FE000E55DFE4F808152DEDF91CF911F910F9111
:101FF0005FCEDF91CF911F910F910895CF92DF9225
:10200000EF92FF920F931F93CF93DF93EC01E8A819
:1020100000E010E0F12CC701002E02C095958795D5
:102020000A94E2F7817021DE1DDE0F5F1F4F08303A
:10203000110589F75C9A5C98FE0180E090E041E030
:1020400050E060E070E0082F22A933A92115310586
:1020500009F046C0A8A92A2F30E0082E02C0359505
:1020600027950A94E2F720FF34C029A930E0082E12
:1020700002C0359527950A94E2F720FD2AC06A012F
:102080007B01082E04C0CC0CDD1CEE1CFF1C0A9446
:10209000D2F79701860100950A2308AB1AC013AA4C
:1020A00012AA6A017B0104C0CC0CDD1CEE1CFF1CD3
:1020B0000A95D2F797018601009528A9202328AB1D
:1020C00022A933A92115310521F02150310933AB63
:1020D00022AB019632968630910509F0B4CF04C048
:1020E0002130310569F7DBCFDF91CF911F910F913F
:1020F000FF90EF90DF90CF9008951F93CF93DF93E1
:10210000EC01EEA5FFA53097E1F089B182FB112724
:1021100010F982FF05C080918106811101C00995E7
:102120001093810619B1111F1127111F41F08091E1
:102130008206811104C0EEA5FFA581E009951093E8
:102140008206DF91CF911F910895FC016281738116
:102150008481958108951F920F920FB60F921124DA
:102160002F933F934F935F936F937F938F939F939F
:10217000AF93BF93EF93FF93EFE3F6E082819381F8
:10218000A481B5810196A11DB11D82839383A4838F
:10219000B583CF0133DF8FE396E0AFDF8FE396E0C7
:1021A000BBDE8FE396E003DEFF91EF91BF91AF912D
:1021B0009F918F917F916F915F914F913F912F915F
:1021C0000F900FBE0F901F9018958CE691E09093A2
:1021D000400680933F060895CB017FC5CB01642F55
:1021E00084C5FC0184859585FC01E05CFF4F20815E
:1021F0003181FC01EE5BFF4F80819181281B390BFF
:102200002F733327C9010895FC0184859585FC014E
:10221000E05CFF4F40815181FC01EE5BFF4F20816C
:1022200031814217530741F00190F081E02DE80F12
:10223000F91F208130E002C02FEF3FEFC901089560
:10224000FC0184859585FC01E05CFF4F4081518154
:10225000FC01EE5BFF4F208131814217530781F073
:10226000A081B181A80FB91F8C91208131812F5F8E
:102270003F4F2F73332731832083282F30E002C054
:102280002FEF3FEFC9010895FC0181A1882329F0B8
:10229000A489B5898C9186FFFBCF11A20895CF93B5
:1022A000DF93FC0126853785D901A05CBF4F8D9156
:1022B0009C91119701968F739927E901CE5BDF4FAF
:1022C0004881598184179507D9F30D90BC91A02DB1
:1022D000A20FB31F6C93A685B785A05CBF4F119664
:1022E0009C938E93A689B7892C9181E090E0078C0E
:1022F00002C0880F991F0A94E2F7282B2C9381E0E3
:1023000081A30488F589E02D80818064808381E049
:1023100090E0DF91CF9108951F920F920FB60F9228
:1023200011242F933F934F938F939F93EF93FF939A
:102330008091C00082FD1CC04091C60080912A0798
:1023400090912B0701968F73992720912C0730913C
:102350002D078217930771F0E0912A07F0912B0760
:10236000E651F94F408390932B0780932A0702C0D0
:102370008091C600FF91EF919F918F914F913F9176
:102380002F910F900FBE0F901F9018951F920F92D4
:102390000FB60F9211242F933F938F939F93EF9338
:1023A000FF932091E6063091E7068091E806909130
:1023B000E9062817390731F48091C1008F7D809399
:1023C000C10014C0E091E806F091E906EA55F94F22
:1023D00020818091E8069091E90601968F739927F4
:1023E0009093E9068093E8062093C600FF91EF9151
:1023F0009F918F913F912F910F900FBE0F901F9043
:102400001895CF92DF92EF92FF92CF93DF93EC017A
:102410006A017B01411581EE580761057105F1F0F4
:10242000EC89FD8981E090E008A002C0880F991F27
:102430000A94E2F7808360E079E08DE390E0A70101
:10244000960175D421503109410951095695479596
:1024500037952795211580E1380790F0EC89FD89A3
:10246000108260E874E88EE190E0A70196015FD4E5
:1024700021503109410951095695479537952795BE
:10248000E889F9893083EA89FB89208319A2EE89DA
:10249000FF89408181E090E09C010C8C02C0220FFA
:1024A000331F0A94E2F7422B4083EE89FF89408173
:1024B0009C010D8C02C0220F331F0A94E2F7422BBD
:1024C0004083EE89FF8940819C010E8C02C0220F5F
:1024D000331F0A94E2F7422B4083EE89FF89208163
:1024E0000F8C02C0880F991F0A94E2F7809582230F
:1024F0008083DF91CF91FF90EF90DF90CF90089590
:10250000109287061092860688EE93E0A0E0B0E075
:102510008093880690938906A0938A06B0938B06D1
:1025200084E891E090938506809384068AEE96E095
:10253000909391068093900686EA96E09093930696
:102540008093920685EC90E0909395068093940694
:1025500084EC90E0909397068093960680EC90E050
:10256000909399068093980681EC90E090939B0657
:1025700080939A0682EC90E090939D0680939C064F
:1025800086EC90E090939F0680939E0684E0809373
:10259000A00683E08093A10687E08093A20685E0F1
:1025A0008093A30681E08093A4060895CF92DF92E2
:1025B000EF92FF920F931F93CF93DF936C01EB0188
:1025C0007A01E60EF71E00E010E00BC06991D6011B
:1025D000ED91FC910190F081E02DC6010995080F65
:1025E000191FCE15DF0591F7C801DF91CF911F911B
:1025F0000F91FF90EF90DF90CF90089561157105D6
:1026000081F0DB010D900020E9F7AD014150510947
:10261000461B570BDC01ED91FC910280F381E02D0C
:10262000099480E090E00895DC01ED91FC91019027
:10263000F081E02D09940F931F93CF93DF93EC016A
:102640006DE0F2DF8C016AE0CE01EEDF9C01200F2D
:10265000311FC901DF91CF911F910F9108950F9301
:102660001F93CF93DF93EC01C9DF8C01CE01E3DF31
:102670009801280F391FC901DF91CF911F910F9148
:1026800008951F920F920FB60F9211242F933F932C
:102690008F939F93AF93BF9380912E0790912F07B5
:1026A000A0913007B091310730913607232F2D5F6D
:1026B0002D3720F40196A11DB11D05C0232F2A57E7
:1026C0000296A11DB11D2093360780932E0790938B
:1026D0002F07A0933007B093310780913207909174
:1026E0003307A0913407B09135070196A11DB11DA4
:1026F0008093320790933307A0933407B093350744
:10270000BF91AF919F918F913F912F910F900FBEED
:102710000F901F901895789484B5826084BD84B51D
:10272000816084BD85B5826085BD85B5816085BDCC
:10273000EEE6F0E0808181608083E1E8F0E01082E5
:10274000808182608083808181608083E0E8F0E026
:10275000808181608083E1EBF0E080818460808310
:10276000E0EBF0E0808181608083EAE7F0E0808147
:1027700084608083808182608083808181608083A7
:102780008081806880831092C1000895833069F051
:1027900028F48130A1F0823011F514C08630B1F0F8
:1027A0008730C1F08430D9F404C0809180008F77E5
:1027B00003C0809180008F7D80938000089584B550
:1027C0008F7702C084B58F7D84BD08958091B0005D
:1027D0008F7703C08091B0008F7D8093B000089503
:1027E000CF93DF9390E0FC01E851FF4F4491FC014F
:1027F000E450FF4F8491882341F190E0880F991FA6
:10280000FC01EC5DFE4F25913491D901865E9E4F0F
:10281000FC0185919491C82FD92F9FB7F8948C9182
:10282000611106C0409584238C938881842308C05D
:10283000623041F4242F209582238C938881842B4D
:10284000888302C0842B8C939FBFDF91CF91089522
:10285000CF93DF93282F30E0F901EC52FF4F8491A2
:10286000F901E851FF4FD491F901E450FF4FC491B1
:10287000CC2381F081118ADFEC2FF0E0EE0FFF1FF7
:10288000E05FFE4F85919491DC018C918D2321E0D6
:1028900030E011F420E030E0C901DF91CF910895DC
:1028A000F894AAC25058BB27AA270ED075C166D18A
:1028B00030F06BD120F031F49F3F11F41EF45BC176
:1028C0000EF4E095E7FB51C1E92F77D180F3BA17F9
:1028D000620773078407950718F071F49EF58FC19E
:1028E0000EF4E0950B2EBA2FA02D0B01B90190012B
:1028F0000C01CA01A0011124FF27591B99F0593F6F
:1029000050F4503E68F11A16F040A22F232F342FB6
:102910004427585FF3CF469537952795A795F04004
:102920005395C9F77EF41F16BA0B620B730B840B19
:10293000BAF09150A1F0FF0FBB1F661F771F881FD1
:10294000C2F70EC0BA0F621F731F841F48F4879529
:1029500077956795B795F7959E3F08F0B3CF939518
:10296000880F08F09927EE0F979587950895D9D08D
:1029700008F481E008950CD00FC107D140F0FED0DB
:1029800030F021F45F3F19F0F0C0511139C1F3C0AC
:1029900014D198F39923C9F35523B1F3951B550B23
:1029A000BB27AA2762177307840738F09F5F5F4F22
:1029B000220F331F441FAA1FA9F333D00E2E3AF063
:1029C000E0E830D091505040E695001CCAF729D07D
:1029D000FE2F27D0660F771F881FBB1F26173707CC
:1029E0004807AB07B0E809F0BB0B802DBF01FF27FC
:1029F00093585F4F2AF09E3F510568F0B6C000C162
:102A00005F3FECF3983EDCF3869577956795B79535
:102A1000F7959F5FC9F7880F911D9695879597F950
:102A20000895E1E0660F771F881FBB1F62177307C9
:102A30008407BA0720F0621B730B840BBA0BEE1FDE
:102A400088F7E095089504D06894B111D9C008952D
:102A5000BCD088F09F5790F0B92F9927B751A0F0BC
:102A6000D1F0660F771F881F991F1AF0BA95C9F722
:102A700012C0B13081F0C3D0B1E00895C0C0672F5B
:102A8000782F8827B85F39F0B93FCCF386957795D2
:102A90006795B395D9F73EF49095809570956195BB
:102AA0007F4F8F4F9F4F0895E89409C097FB3EF4E6
:102AB00090958095709561957F4F8F4F9F4F99238B
:102AC000A9F0F92F96E9BB279395F6958795779509
:102AD0006795B795F111F8CFFAF4BB0F11F460FFC9
:102AE0001BC06F5F7F4F8F4F9F4F16C0882311F021
:102AF00096E911C0772321F09EE8872F762F05C035
:102B0000662371F096E8862F70E060E02AF09A95CF
:102B1000660F771F881FDAF7880F9695879597F9C4
:102B20000895990F0008550FAA0BE0E8FEEF16165E
:102B30001706E807F907C0F012161306E407F507B1
:102B400098F0621B730B840B950B39F40A2661F025
:102B5000232B242B252B21F408950A2609F4A140C8
:102B6000A6958FEF811D811D089597F99F6780E8D5
:102B700070E060E008959FEF80EC089500240A94CF
:102B80001616170618060906089500240A94121648
:102B90001306140605060895092E0394000C11F47B
:102BA000882352F0BB0F40F4BF2B11F460FF04C028
:102BB0006F5F7F4F8F4F9F4F089557FD9058440F81
:102BC000551F59F05F3F71F04795880F97FB991F8C
:102BD00061F09F3F79F08795089512161306140649
:102BE000551FF2CF4695F1DF08C0161617061806D6
:102BF000991FF1CF86957105610508940895E894B1
:102C0000BB2766277727CB0197F908958ADF08F459
:102C10008FEF08950BD0C0CFB1DF28F0B6DF18F0EA
:102C2000952309F0A2CFA7CF1124EACFC6DFA0F3E6
:102C3000959FD1F3950F50E0551F629FF001729F51
:102C4000BB27F00DB11D639FAA27F00DB11DAA1F70
:102C5000649F6627B00DA11D661F829F2227B00DBD
:102C6000A11D621F739FB00DA11D621F839FA00D48
:102C7000611D221F749F3327A00D611D231F849F98
:102C8000600D211D822F762F6A2F11249F575040EF
:102C90008AF0E1F088234AF0EE0FFF1FBB1F661F8A
:102CA000771F881F91505040A9F79E3F510570F043
:102CB0005CCFA6CF5F3FECF3983EDCF3869577952B
:102CC0006795B795F795E7959F5FC1F7FE2B880F3E
:102CD000911D9695879597F90895F999FECF92BD24
:102CE00081BDF89A992780B50895262FF999FECFCE
:102CF0001FBA92BD81BD20BD0FB6F894FA9AF99A19
:102D00000FBE01960895AA1BBB1B51E107C0AA1F65
:102D1000BB1FA617B70710F0A61BB70B881F991F7C
:102D20005A95A9F780959095BC01CD010895A1E22F
:102D30001A2EAA1BBB1BFD010DC0AA1FBB1FEE1F35
:102D4000FF1FA217B307E407F50720F0A21BB30B80
:102D5000E40BF50B661F771F881F991F1A9469F7FC
:102D600060957095809590959B01AC01BD01CF0158
:102D70000895052E97FB16F4009406D057FD0CD04D
:102D8000D6DF07FC09D07EF490958095709561950B
:102D90007F4F8F4F9F4F08955095409530952195C7
:102DA0003F4F4F4F5F4F0895A29FB001B39FC001A7
:102DB000A39F01D0B29F700D811D1124911D089514
:102DC000F3DFB7FF0895821B930B0895EDDFA59FF6
:102DD000900DB49F900DA49F800D911D1124089516
:102DE000B7FFF4CFF3DF821B930B0895EE0FFF1FA5
:0C2DF0000590F491E02D0994F894FFCFB9
:102DFC0001000000000000000000000000000014B2
:102E0C00000002000106FF00040405030400005545
:102E1C0021E507E5559A15B53B121F050403020180
:102E2C00000001020406050307636C656172546FB0
:102E3C005B5D3D7B20002C20002C202000207D3B66
:102E4C00200073746172740000000020C81F7FB8EA
:102E5C0000101D0010FF7F00000000002B0E2A0E3A
:102E6C00200E210E220E230E250E260E270E280EC6
:102E7C00000000004F11D612F11020110411441162
:00000001FF
